S01D000062696E2F6F70656E626C745F73746D3332683734332E737265638D
S3150800000000000220050400085504000855040008ED
S3150800001055040008550400085504000800000000AF
S315080000200000000000000000000000005504000861
S31508000030550400080000000055040008715C00081B
S31508000040550400085504000855040008550400081E
S31508000050550400085504000855040008550400080E
S3150800006055040008550400085504000855040008FE
S3150800007055040008550400085504000855040008EE
S3150800008055040008550400085504000855040008DE
S3150800009055040008550400085504000855040008CE
S315080000A055040008550400085504000855040008BE
S315080000B055040008550400085504000855040008AE
S315080000C0550400085504000855040008550400089E
S315080000D0550400085504000855040008550400088E
S315080000E055040008550400080000000055040008DF
S315080000F0550400085504000855040008550400086E
S31508000100550400085504000855040008550400085D
S31508000110550400085504000855040008550400084D
S31508000120550400085504000855040008550400083D
S31508000130550400085504000855040008550400082D
S3150800014000000000000000000000000000000000A1
S31508000150550400085504000855040008550400080D
S3150800016055040008550400085504000855040008FD
S31508000170550400085504000855040008000000004E
S3150800018055040008550400085504000855040008DD
S3150800019055040008550400085504000855040008CD
S315080001A055040008550400085504000855040008BD
S315080001B055040008550400085504000855040008AD
S315080001C0550400085504000855040008550400089D
S315080001D0550400085504000855040008550400088D
S315080001E0550400085504000855040008550400087D
S315080001F0550400085504000855040008550400086D
S31508000200550400085504000855040008550400085C
S31508000210550400085504000855040008550400084C
S31508000220550400085504000855040008000000009D
S31508000230550400085504000800000000550400088D
S31508000240550400085504000855040008550400081C
S31508000250550400085504000855040008550400080C
S3150800026055040008550400085504000855040008FC
S31508000270550400085504000855040008000000004D
S31508000280550400085504000855040008000000003D
S30D080002900000000055040008F7
S3150800029810B5054C237833B9044B13B10448AFF3AA
S315080002A800800123237010BDF00400200000000020
S315080002B8985C000808B5034B1BB103490348AFF31C
S315080002C8008008BD00000000F4040020985C0008BF
S315080002D870B50D4E0D4D761BB61006D000240134A8
S315080002E855F8043B9847A642F9D1094E094D761B9D
S315080002F805F0CEFCB61006D00024013455F8043BA8
S315080003089847A642F9D170BD105F0008105F00082B
S31508000318185F0008105F0008024B13B1024800F086
S3150800032805B870470000000041030008002301468D
S315080003381A46184600F01EB838B50A4C0A4D641B0A
S31508000348A4100AD004F18043013B05EB8305013C60
S3150800035855F804399847002CF9D1BDE8384005F016
S315080003689DBC00BF1C5F0008185F0008704700BFE7
S31508000378704700BF2DE9F0411E4C05462068904697
S315080003881F460E46FFF7F2FF1B4B1A68D2F848318C
S3150800039833B35A6820681F2A27DC4DB9911C0132E5
S315080003A85A6043F82160FFF7E3FF0020BDE8F081B3
S315080003B803EB82010124C1F8888004FA02FED3F807
S315080003C88841022D44EA0E0CC3F888C1C1F80871A1
S315080003D8E4D1D3F88C114EEA0104C3F88C41DDE761
S315080003E802F5A673C2F84831D3E7FFF7C1FF4FF005
S315080003F8FF30DBE728040020FC5C0008DFF834D06F
S31508000408002103E00C4B5B58435004310B480C4B56
S3150800041842189A42F6D30B4A02E0002342F8043BF4
S31508000428094B9A42F9D303F09FFDFFF751FF00F0F5
S3150800043843FA7047000002201C5F000800000020ED
S31508000448F0040020F004002034190020FEE708B55F
S3150800045800F57171D0F8040403F00DFE08BD08B55F
S31508000468C1EBC10293000344D3F80822D0F8040468
S3150800047803F02FFE08BD08B5C1EBC102930003447B
S315080004889A6CD0F8040403F06EFE08BD08B5D0F8D7
S31508000498040403F013FF08BD10B50446C3684BB13E
S315080004A8022B01D1012106E09121074804F0BEFD7F
S315080004B8012100E00021D4F8040403F0E8FED4F88A
S315080004C8040403F0BCFE10BD005D000810B5044620
S315080004D8D0F8040403F0DEFE2268D2F8003E43F0A2
S315080004E80103C2F8003E236A23B1044A136943F09C
S315080004F80603136100F000FB10BD00BF00ED00E025
S3150800050810B5044600F0F9FAD4F8040403F0CBFE53
S3150800051810BD08B5D0F8040403F0E0FE08BD08B518
S31508000528D0F8040403F0D8FE08BD10B50446012027
S3150800053800F0E1FAD4F8040403F0D2FE10BD10B5B1
S315080005480446002000F0D7FAD4F8040403F0CAFEDB
S3150800055810BD000003780BB10020704710B503469C
S315080005681748C0F80434C3F8C002164B03600923B9
S3150800057843600222C2600023036182610122C261CC
S31508000588036243628362C362036301F00FFF80B9A3
S315080005980B4C8021204600F0DFFB40220021204634
S315080005A800F0B6FB80220121204600F0B1FB0020AE
S315080005B810BD4FF49371044804F038FDE8E700BF0E
S315080005C8D012002000000840005D0008D0F8C032AC
S315080005D811F0800F08D101F07F01C1EBC1018A0033
S315080005E8134493F8FE01704701F07F01C1EBC1017E
S315080005F88A00134493F83E00704708B5D0F8C0023D
S3150800060802F0C4FB08BD022807D8DFE800F0020696
S31508000618040000207047012070470220704708B57B
S31508000628D0F8C00201F09CFFFFF7EDFF08BD08B53A
S31508000638D0F8C00201F053FFFFF7E5FF08BD08B57B
S31508000648D0F8C00201F06CFFFFF7DDFF08BD10B552
S315080006581C4613462246D0F8C00202F0F3FAFFF702
S31508000668D2FF10BD08B5D0F8C00202F02BFBFFF781
S31508000678CAFF08BD08B5D0F8C00202F0BAFBFFF7F2
S31508000688C2FF08BD08B5D0F8C00202F0F3FBFFF7B1
S31508000698BAFF08BD08B5D0F8C00202F0BFFAFFF7DE
S315080006A8B2FF08BD08B5D0F8C00202F078FBFFF71C
S315080006B8AAFF08BD08B5D0F8C00202F039FBFFF753
S315080006C8A2FF08BD014B1880704700BF0C05002023
S315080006D808B505F0BDFA0E4B1B6898420FD30D4BAB
S315080006E81B786BB90B4B01221A700B4B80229A6147
S315080006F805F0AEFA094B1B881844054B186008BD67
S31508000708044B00221A70044B4FF400029A61EFE773
S31508000718100500200E050020000402580C050020CC
S31508000728024B4FF400029A61704700BF0004025852
S3150800073808B5574A136823F00F0343F004031360F8
S31508000748136803F00F03042B40F09C80514AD368C2
S3150800075823F0070343F00203D360936943F4404345
S3150800076893614D4B1A6842F480221A601A6842F45B
S3150800077880321A60484B1B6813F4003FFAD0464B80
S315080007889A6A22F0030242F002029A62DA6A42F48C
S315080007988032DA62DA6A42F40032DA62DA6A22F017
S315080007A80C0242F00402DA62DA6A22F00202DA621B
S315080007B89A6A22F47C7242F040029A621A6B3749A6
S315080007C8114040F2DF120A431A631A6B22F47E427A
S315080007D842F400721A631A6B22F4FE0242F4981263
S315080007E81A631A6B22F0FE4242F080721A631A687C
S315080007F842F080721A60284B1B6813F0007FFAD003
S31508000808254B9A6922F00F0242F008029A611A6982
S3150800081822F0070242F003021A619A6922F470620A
S315080008289A619A6922F00F0242F008029A61DA6917
S3150800083822F0700242F04002DA61DA6922F4E062D4
S3150800084842F48062DA619A6922F0700242F0400244
S315080008589A611A6A22F0700242F040021A62104936
S315080008680A6822F007020A601A6D22F040521A65D1
S315080008785A6D22F4401242F480125A65094800F06B
S3150800088825FC08BD6721084804F0D0FB5EE700BFD1
S3150800089800200052004802580044025800FEFFFF94
S315080008A85444025800389C1C0C5D000808B500F032
S315080008B8C5FAFFF73DFF08BD08B5FFF7F7FF04F0CF
S315080008C84BFB04F057FBFCE72DE9F0418EB0514C81
S315080008D8D4F8F43043F00203C4F8F430D4F8F4300A
S315080008E803F002030793079BD4F8E03043F00103AB
S315080008F8C4F8E030D4F8E03003F001030693069B09
S31508000908D4F8E03043F00203C4F8E030D4F8E03015
S3150800091803F002030593059BD4F8E03043F004037B
S31508000928C4F8E030D4F8E03003F004030493049BD9
S31508000938D4F8E03043F00803C4F8E030D4F8E030DF
S3150800094803F008030393039BD4F8E83043F48023A1
S31508000958C4F8E830D4F8E83003F480230293029BFD
S31508000968D4F8EC3043F48073C4F8EC30D4F8EC309F
S3150800097803F480730193019B802308930123099349
S3150800098800250A950B950C95234F08A9384601F0BA
S315080009983DFC4FF40053089309950C9508A91F4880
S315080009A801F034FC4FF44078CDF8208002260996E9
S315080009B80A950B950C9507230D9308A9184801F075
S315080009C825FCCDF8208009960A960B950C950923DF
S315080009D80D9308A9384601F019FC4FF4C05308933B
S315080009E8099603230A930B950C950A230D9308A9D0
S315080009F80C4801F00BFCD4F8D83043F00063C4F86F
S31508000A08D830D4F8D83003F000630093009B0EB0B2
S31508000A18BDE8F0810044025800040258000802584C
S31508000A28000C02580000025810B502F075FE214C59
S31508000A384FF40003A361204801F0FCFA1F4801F0AF
S31508000A48F9FA204601F0F6FA1D4801F0F3FA1D4BAB
S31508000A58D3F8D82022F00062C3F8D820D3F8EC20BF
S31508000A6822F48072C3F8EC20D3F8E82022F4802216
S31508000A78C3F8E820D3F8E02022F00802C3F8E020FB
S31508000A88D3F8E02022F00402C3F8E020D3F8E020E7
S31508000A9822F00202C3F8E020D3F8E02022F001028F
S31508000AA8C3F8E020D3F8F42022F00202C3F8F420B1
S31508000AB810BD00BF00040258000C0258000802586E
S31508000AC8000002580044025808B5054B1B6913F480
S31508000AD8005F03D1FFF724FE012008BD0020FCE7CC
S31508000AE80008025808B56420FFF7ECFD08BD08B5EC
S31508000AF8FFF7EEFD08BD704770477047202303804F
S31508000B0800487047640400200A2303800048704799
S31508000B188404002008B590F89C32032B01D00020E5
S31508000B2808BD04F02FFCFAE708B504F02BFC0020F2
S31508000B3808BD08B5084604F059FC002008BD0000A1
S31508000B4808B50B7813F0600F06D14B780A2B14D02A
S31508000B580B2B17D0062B01D0002008BD4B881B0A83
S31508000B68212B04D00B49172203F028FFF4E7CA887B
S31508000B78172A28BF17220849F6E70122074903F06A
S31508000B881DFFE9E78B7813B9044A1360E4E703F015
S31508000B98DBFBE1E76D04002076040020140500203D
S31508000BA810B504468121FFF75DFD01212046FFF7B0
S31508000BB859FD002010BD000010B504464023022246
S31508000BC88121FFF744FD4023022201212046FFF731
S31508000BD83EFD4023034A01212046FFF76BFD00200E
S31508000BE810BD00BFD816002000487047D816002048
S31508000BF812230B8000487047AC04002004230B809E
S31508000C0800487047C00400200023934216D230B427
S31508000C180BE0373401F8134000015C000134002565
S31508000C280D550133DBB2934206D2040F092CF0D8CE
S31508000C38303401F81340EFE730BC704770470000BE
S31508000C4838B50A4B186804331C6804331B68C0187F
S31508000C5800D138BD064D0822A91CFFF7D5FF042286
S31508000C6805F112012046FFF7CFFFF2E700E8F11F6A
S31508000C78C404002008B51A230B80FFF7E1FF0148D2
S31508000C8808BD00BFC404002008B50A4628B90549A6
S31508000C98054803F078FE034808BD0249024803F0F0
S31508000CA872FEF8E718170020445D000810B5044CD2
S31508000CB80A462146034803F066FE204610BD00BFD3
S31508000CC818170020345D000808B50A4628B90549EA
S31508000CD8054803F058FE034808BD0249024803F0D0
S31508000CE852FEF8E718170020145D000808B50A46EA
S31508000CF828B90549054803F046FE034808BD0249D0
S31508000D08024803F040FEF8E7181700201C5D0008A3
S31508000D1830B40468606A29B940EA0240A062002033
S31508000D2830BC70470D46A36A00EB13400023691EC2
S31508000D388B4209D203F1400104EB8101496800EBB3
S31508000D4811400133DBB2F2E740EA024005F13F0100
S31508000D5804EB81014860E2E703685962002070479E
S31508000D68024603680121C0F8FC13002082F8F40340
S31508000D789A6942F000629A61596D024A0A435A65AD
S31508000D88704700BF030000107047000010B5164BE7
S31508000D986FF00042DA670024DC674FF0FF32C3F8C9
S31508000DA88020C3F88040C3F88420C3F88440C3F879
S31508000DB88820C3F88840C3F88C20C3F88C40C3F849
S31508000DC89020C3F89040C3F89420C3F89440C3F819
S31508000DD89820C3F89840C3F89C20C3F89C40FFF7AE
S31508000DE823FE204610BD00BF00440258104B1B784E
S31508000DF80BB90120704710B504464FF47A70B0FB5A
S31508000E08F3F30C4A1068B0FBF3F000F09DF868B9E4
S31508000E180F2C01D901200AE0002221464FF0FF30A5
S31508000E2800F060F8044B1C60002000E0012010BDAB
S31508000E38DE040020E4040020E004002010B50320A6
S31508000E4800F03EF800F048F90F498B69C3F303230D
S31508000E580E4AD35C03F01F03D8408B6903F00F03CF
S31508000E68D35C03F01F0320FA03F3094A1360094BFE
S31508000E7818600020FFF7BAFF10B10124204610BDFC
S31508000E880446FFF721FDF9E700440258A85D000863
S31508000E98E8040020E404002038B5044604F0E0FE1F
S31508000EA80546B4F1FF3F02D0044B1B781C4404F0F6
S31508000EB8D7FE401BA042FAD338BD00BFDE04002087
S31508000EC80649CB6823F4E0631B041B0C000200F4F4
S31508000ED8E0600343024A1A43CA60704700ED00E01F
S31508000EE80000FA0530B4154BDB68C3F30223C3F1D7
S31508000EF80704042C28BF04241D1D062D01D9033B0D
S31508000F0800E000234FF0FF3505FA04F421EA04014E
S31508000F18994005FA03F322EA03031943002805DB77
S31508000F280901C9B2064B195430BC704700F00F00C6
S31508000F380901C9B2034B1954F6E700BF00ED00E0F2
S31508000F4800E400E014ED00E00138B0F1807F0AD231
S31508000F58064B5860064AF02182F82310002098604C
S31508000F6807221A6070470120704700BF10E000E0AA
S31508000F7800ED00E038B5036813F0010F40F08C80E7
S31508000F880D4604460368454A1A408B6809690B43A7
S31508000F9869690B43E9690B4313430360EB684268C5
S31508000FA822F4405213434360AB69826822F44072C4
S31508000FB8134383603A4B984216D03A4B98421CD052
S31508000FC8394B98421DD0394B98421ED0384B984217
S31508000FD81FD0384B984220D0374B984221D0374BF0
S31508000FE8984222D001204EE0354802F007FE002834
S31508000FF848D06A68EAB9012045E0324802F0FEFDA1
S31508001008F5E7304802F0FAFDF1E72E4802F0F6FD5A
S31508001018EDE72C4802F0F2FDE9E7294802F0EEFD73
S31508001028E5E7284802F0EAFDE1E7264802F0E6FD8A
S31508001038DDE72B68E9690B2B2CD8B1F5004F0DD0E5
S31508001048DBB2214951F82330B0FBF3F303EB520323
S31508001058B3FBF2F39BB2E360002014E0DBB21A4953
S3150800106851F82330B0FBF3F0530803EB4000B0FB0C
S31508001078F2F34FF6F0721A40C3F342031343E360E0
S31508001088002000E00120E26A22F00F022B881343B1
S31508001098E36202E00020F6E7012038BDF369FFEFB6
S315080010A8001001400044004000480040004C004041
S315080010B8005000400014014000780040007C0040C1
S315080010C80803000708000007585D0008014B186068
S315080010D8704700BFE4040020724B1B6903F038030D
S315080010E8102B00F0DB80182B10D00BB16E48704718
S315080010F86C4B1B6813F0200F00F0D280694B1868F8
S31508001108C0F3C100694B23FA00F07047654A916A33
S3150800111801F00301906AC0F30510D36A03F00103CE
S31508001128526BC2F3CC0203FB02F307EE903AF8EED1
S31508001138677A002800F0B580012966D0F9B1022936
S3150800114800F08F8007EE100AF8EE476A9FED586A96
S3150800115886EE267A534B1B6BC3F3080306EE903AC2
S31508001168F8EE666A9FED536A67EE867A76EEA77A90
S31508001178F7EE006A77EEA67A27EE277A61E0494BFA
S315080011881B6813F0200F23D046490A68C2F3C10228
S31508001198464BD34007EE103AF8EE476A07EE100AB0
S315080011A8B8EE476A86EE867A0B6BC3F3080306EE33
S315080011B8903AF8EE666A9FED3F6A67EE867A76EEAB
S315080011C8A77AF7EE006A77EEA67A27EE277A38E046
S315080011D807EE100AF8EE476A9FED376A86EE267A12
S315080011E8304B1B6BC3F3080306EE903AF8EE666AB3
S315080011F89FED306A67EE867A76EEA77AF7EE006A8A
S3150800120877EEA67A27EE277A1BE007EE100AF8EE9D
S31508001218476A9FED276A86EE267A224B1B6BC3F32D
S31508001228080306EE903AF8EE666A9FED226A67EEBC
S31508001238867A76EEA77AF7EE006A77EEA67A27EE2A
S31508001248277A184B1B6BC3F34623013307EE903AEC
S31508001258F8EE677AC7EE276AFCEEE67A17EE900A82
S31508001268704707EE100AF8EE476A9FED146A86EE8D
S31508001278267A0C4B1B6BC3F3080306EE903AF8EE76
S31508001288666A9FED0C6A67EE867A76EEA77AF7EEB7
S31508001298006A77EEA67A27EE277AD2E708487047D3
S315080012A8024870470044025800093D000090D003E0
S315080012B80024744A000000390024744C0024F44AB7
S315080012C800127A0008B5FFF707FF0B4A9369C3F3BC
S315080012D803230A49CB5C03F01F0320FA03F3926938
S315080012E802F00F02885C00F01F0023FA00F0044A97
S315080012F81060044A136008BD00440258A85D000837
S31508001308E8040020E4040020002301330C4A934231
S3150800131811D80269002AF8DA036943F00103036160
S3150800132800230133064A934207D8026912F0010FCF
S31508001338F7D100207047032070470320704700BF85
S31508001348400D030084B010B5044603A880E80E00D3
S31508001358089B012B1DD1A36B23F48033A363E26892
S315080013681A4B1340E360E36823F44013E3600F9BCA
S31508001378012B09D02046FFF7C7FF069B012B1BD078
S31508001388BDE8104004B07047E36843F48013E3608F
S31508001398F0E7E36843F04003E3602046FFF7B4FF4D
S315080013A80C9B23B9A36B43F48033A363E5E7A36BCC
S315080013B823F48033A363E0E7A36843F00603A36036
S315080013C8A36843F02003A360DAE700BFBFFFBDFFA9
S315080013D8022A0AD00921C26822F47052C260C36878
S315080013E843EA8123C36000207047274B0B44274AEA
S315080013F8934237D9264B0B44264A934234D9264B6F
S315080014080B44264A934231D9254B0B4402F5C3327D
S31508001418A03293422CD9234B0B44234A934229D909
S31508001428224B0B4402F5922202F57872934223D98D
S315080014381F4B0B4402F5C32202F5207293421DD9AD
S315080014481C4B0B4402F5B71202F55872934217D98A
S31508001458194B0B4402F5122202F5F862934211D889
S315080014680721B8E70F21B6E70E21B4E70D21B2E741
S315080014780C21B0E70B21AEE70A21ACE70921AAE758
S315080014880821A8E70621A6E7405327FFFF340C00E2
S31508001498401E1BFF3F420F0000DC0BFF7F4F120068
S315080014A8808CF9FE60B6E5FE5FE3160000D3CEFE33
S315080014B8C05BB3FE00CA91FEE05459FE836843F048
S315080014C80103836000207047836823F00103836063
S315080014D80020704708B5C36823F0C043C3600129D4
S315080014E809D069B9C36843F08043C3603220FFF75F
S315080014F8D3FC002008BDC36843F00053C360F5E772
S315080015080120F7E7890141F0200101610023013331
S31508001518054A934205D8026912F0200FF7D1002030
S3150800152870470320704700BF400D0300102303616E
S3150800153800230133054A934205D8026912F0100FB1
S31508001548F7D1002070470320704700BF400D0300FD
S31508001558D0F800381943C0F8001800207047000072
S3150800156884B0F8B5044607A880E80E002546002387
S315080015780E2B07D803F1400204EB820200215160C2
S315080015880133F5E7119B23BBD4F8043843F002036B
S31508001598C4F80438A36B23F40013A363236843F041
S315080015A840032360236843F0800323600023C4F8BC
S315080015B8003E04F50066D4F80038C4F800380C9BD9
S315080015C8012B10D1099B4BB900212046FFF7C0FF14
S315080015D80DE0A36B43F40013A363E7E70121204654
S315080015E8FFF7B6FF03E003212046FFF7B1FF1021F6
S315080015F82046FFF787FF074600B101272046FFF771
S3150800160895FF00B10127002333617361F3610AE08E
S31508001618C3B94FF00060C2F8000900220A614FF604
S315080016287F328A600133079A9A4210D905EB43122A
S3150800163802F51061D2F800090028E9DB0020C2F893
S315080016480009EAE74FF09040C2F80009E5E70023E9
S315080016580AE0C3B94FF00060C2F8000B00220A611D
S315080016684FF67F328A600133079A9A4210D905EBFA
S31508001678431202F53061D2F8000B0028E9DB002096
S31508001688C2F8000BEAE74FF09040C2F8000BE5E70E
S31508001698336923F4807333610023A3616FF08043B1
S315080016A863610A9B1BB9A36943F01003A361A26986
S315080016B80A4B1343A3610D9B1BB1A36943F00803A7
S315080016C8A361119B012B04D03846BDE8F84004B045
S315080016D87047A269024B1343A361F5E700383C80BB
S315080016E804000040D0F8083813F0060305D0062B86
S315080016F818BF022B03D102207047002070470F201D
S315080017087047000070B40B784A78012A20D0D0F8C0
S315080017181C2803F00F060124B44042EA0442C0F824
S315080017281C2800EB4310D0F8003B13F4004F0CD1EB
S31508001738D0F8002B8B68C3F30A03C97843EA8143B8
S315080017481343134A1A43C0F8002B002070BC70478D
S31508001758D0F81C4803F00F06B24092B22243C0F8EC
S315080017681C2800EB4310D0F8002912F4004FECD1DE
S31508001778D0F800498A68C2F30A02C97842EA81425F
S3150800178842EA8353234302491943C0F80019DCE7A0
S315080017980080001070B40B784A78012A1FD0D0F858
S315080017A83C5803F00F06012404FA06F625EA06450E
S315080017B8C0F83C58D0F81C58097801F00F018C403D
S315080017C825EA0444C0F81C4800EB4310D0F8002B5F
S315080017D8124B1340C0F8003B002070BC7047D0F885
S315080017E83C6803F00F0402FA04F4A4B226EA0404D7
S315080017F8C0F83C48D0F81C48097801F00F018A401F
S3150800180892B224EA0202C0F81C2800EB4310D0F86A
S315080018180039034A1A40C0F80029DDE70078F3EFD3
S31508001828007833EC70B40B784C78012C24D000EB94
S31508001838431000F530631D693E4C2C401C611D6938
S315080018483D4C2C401C614C690CB18C684C611C6978
S3150800185844F400241C611C698D68C5F312052C43E1
S315080018681C61012A61D0D0F8003B43F00443C0F854
S31508001878003B002070BC70474C695CBB00EB431406
S31508001888D4F810692C4D3540C4F81059D4F81059B5
S3150800189845F40025C4F81059D4F81069254D354083
S315080018A8C4F81059012A31D000EB4313D3F800299C
S315080018B842F00442C3F800294B69002BD9D0D0F866
S315080018C83428097801F00F040121A1400A43C0F819
S315080018D83428CEE700EB431404F510642669154D41
S315080018E8354025612669144D354025614E698D6850
S315080018F8AE4200D94D61256945F40025256125695B
S315080019084E69C6F3120635432561CBE70A691AB14B
S3150800191800EB4311C1F8142900EB4310D0F800294D
S3150800192842F00442C0F80029A3E7CA68002A9AD0F8
S315080019385A6198E70000F8FFFFFF07E070B49DF8C2
S315080019480C4064B903339E08B44208D200EB02334C
S3150800195803F5805351F8045B1D600134F4E7002051
S3150800196870BC7047F0B583B00B784C78012C29D039
S3150800197800EB431303F5306426697C4D3540256131
S3150800198826697B4D354025614D69002D40F0BF809D
S3150800199825698E68C6F3120635432561256945F417
S315080019A800252561012A00F0C780CA78012A00F0B7
S315080019B8C980D3F8002B42F00442C3F8002B002054
S315080019C803B0F0BD4C6974BB00EB4314D4F8106936
S315080019D8674D3540C4F81059D4F8105945F4002510
S315080019E8C4F81059D4F81069604D3540C4F8105930
S315080019F8012A4AD000EB4313D3F8004944F00444BB
S31508001A08C3F80049CC78012C68D04B69002BD6D08E
S31508001A18D0F83428097801F00F040121A1400A43B7
S31508001A28C0F83428CBE700EB4314D4F810694F4DB7
S31508001A383540C4F81059D4F810694D4D3540C4F8E6
S31508001A481059D4F810694D698F683D44013DB5FBB6
S31508001A58F7F5484F07EAC5453543C4F81059D4F889
S31508001A6810594E69C6F312063543C4F8105904F5D9
S31508001A781064CD78012DBBD1256925F0C0452561AF
S31508001A88256945F000552561B2E70A691AB100EBE0
S31508001A984314C4F81429CA78012A08D000EB43135A
S31508001AA8D3F8002942F00442C3F8002987E7D0F89A
S31508001AB8082812F4807F08D100EB4311D1F80029D1
S31508001AC842F00052C1F80029E8E700EB4311D1F8C3
S31508001AD8002942F08052C1F80029DFE7D0F8084803
S31508001AE814F4807F0CD1D3F8004944F00054C3F8A5
S31508001AF8004900928B8A0A78C968FFF71FFF5EE7D4
S31508001B08D3F8004944F08054C3F80049F1E78E68D1
S31508001B183544013DB5FBF6F52669164F07EAC5476C
S31508001B283E43266127698E68ADB206FB05F5C5F3FF
S31508001B3812053D43256135E7CA68002A3FF435AFE3
S31508001B48626132E7D0F8082812F4807F06D1D3F804
S31508001B58002B42F00052C3F8002B2AE7D3F8002BD3
S31508001B6842F08052C3F8002B23E700BF0000F8FFB5
S31508001B78FFFF07E00000F81F03329208002393428C
S31508001B880CD210B400F58054246841F8044B01338C
S31508001B989342F7D308465DF8044B704708467047E2
S31508001BA80B784A78012A14D000EB4310D0F8002B9A
S31508001BB8002A06DB2BB1D0F8003B23F08043C0F897
S31508001BC8003BD0F8003B43F40013C0F8003B002064
S31508001BD8704700EB4310D0F80029002A06DB2BB122
S31508001BE8D0F8003923F08043C0F80039D0F8003916
S31508001BF843F40013C0F80039E9E70B784A78012A54
S31508001C080ED000EB4310D0F8003B23F40013C0F8BD
S31508001C18003BCB78023BDBB2012B15D90020704775
S31508001C2800EB4310D0F8003923F40013C0F8003944
S31508001C38CB78023BDBB2012BF0D8D0F8003943F059
S31508001C488053C0F80039E9E7D0F8003B43F08053E1
S31508001C58C0F8003BE2E738B50546044600220E2AD6
S31508001C6809D804EB42134FF67F31C3F80819C3F8AD
S31508001C78081B0132F3E70022C5F81028C5F814280E
S31508001C88C5F81C282846FFF751FC034608B118462C
S31508001C9838BD10212846FFF735FC0346F7E7D0F884
S31508001CA8003823F4FE63C0F80038D0F80038090174
S31508001CB801F4FE610B43C0F800380020704708B5E8
S31508001CC8D0F8043823F00203C0F804380320FFF7D5
S31508001CD8E3F8002008BD08B5D0F8043843F0020335
S31508001CE8C0F804380320FFF7D7F8002008BD426972
S31508001CF8806910407047D0F8183800F50060C06948
S31508001D081840000C7047D0F8183800F50060C0690C
S31508001D18184080B2704700EB4111D1F8082B00F53E
S31508001D28006040691040704710B4D0F81048D0F8E1
S31508001D38343801F00F02D340DB01DBB2234300EB52
S31508001D48411000F51060806818405DF8044B70472C
S31508001D58406900F001007047D0F80029054B134088
S31508001D68C0F80039D0F8043843F48073C0F804384A
S31508001D780020704700F8FFFF10B4046C154B9C420E
S31508001D8803D9D0F8003B002B16DB0024C0F8104B0B
S31508001D98D0F8104B44F40024C0F8104BD0F8104B78
S31508001DA844F01804C0F8104BD0F8104B44F0C0445F
S31508001DB8C0F8104B012903D000205DF8044B704782
S31508001DC8C0F8142BD0F8003B43F08023C0F8003B3A
S31508001DD8F2E700BF0A30544F144BDB6813F0010FC3
S31508001DE809D0124B124A5A6002F188325A60DB68E7
S31508001DF813F0010F14D10D4BD3F80C3113F0010F62
S31508001E0810D00A4B0A4AC3F8042102F18832C3F8EB
S31508001E180421D3F80C3113F0010F05D100207047BF
S31508001E2801207047002070470120704700200052A3
S31508001E38230167450D4BDA6842F00102DA60DB6870
S31508001E4813F0010F0DD0094BD3F80C2142F001020B
S31508001E58C3F80C21D3F80C3113F0010F03D0002076
S31508001E687047012070470120704700BF00200052C4
S31508001E78F8B505460E4603F0F3FE0746012E09D0C7
S31508001E88364C17E003F0ECFEC01BA84260D88DB9A3
S31508001E9803204EE004240DE0314BD3F8103124EA30
S31508001EA8030333F000430CBF012300236BB1B5F1DC
S31508001EB8FF3FE7D134F00403EED1294B1B6934EA16
S31508001EC803030CBF01230023F0E7012E1CD0244B83
S31508001ED8D3F8103123F0684323F480135B0C5B04B2
S31508001EE843F0004333F0024217D1012E25D01C4B8C
S31508001EF8D3F8103113F4803F2ED0194B4FF48032A3
S31508001F08C3F81421002014E0154B1B6923F0684315
S31508001F1823F480135B0C5B04E4E712498A691A43C5
S31508001F288A61002B06DA23F000430D4AC2F81431F9
S31508001F380120F8BD0A4A5361FAE7094B1B6913F4ED
S31508001F48803F07D0064B4FF480325A610020F0E7ED
S31508001F580320EEE70020ECE70020EAE7040000800B
S31508001F6800200052181900202C4B1B7D012B51D03C
S31508001F7870B50C461546294B01221A7501F17841A8
S31508001F88B1F5801F38D21646244B00229A6131468D
S31508001F984CF25030FFF76CFF034640BB012E2DD09C
S31508001FA81F4AD2F80C3143F00203C2F80C31BFF3CA
S31508001FB86F8FBFF34F8F082355F8042B44F8042B6B
S31508001FC8013B13F0FF03F7D1BFF36F8FBFF34F8FB2
S31508001FD831464CF25030FFF74BFF0346012E13D01B
S31508001FE80F49D1F80C2122F00202C1F80C210B4A3C
S31508001FF800211175184670BD0226C5E7084AD36838
S3150800200843F00203D360D2E70549CA6822F0020200
S31508002018CA60ECE702231846704700BF1819002063
S3150800202800200052024AD36843F08073D360704791
S31508002038004802586A4B984222D06A4B98422FD0D9
S31508002048694B98423CD0694B984249D0684B9842AC
S3150800205856D0684B984263D0674B984270D0674B06
S3150800206898427DD0664B984200F08A80654B984224
S3150800207800F09680644B984200F0A28001207047D1
S3150800208803F58843D3F8882042F00102C3F888206C
S31508002098D3F8882022F00102C3F888200020704768
S315080020A803F58043D3F8882042F00202C3F8882053
S315080020B8D3F8882022F00202C3F888200020704747
S315080020C803F57053D3F8882042F00402C3F8882031
S315080020D8D3F8882022F00402C3F888200020704725
S315080020E803F56053D3F8882042F00802C3F888201D
S315080020F8D3F8882022F00802C3F888200020704701
S3150800210803F55053D3F8882042F01002C3F8882004
S31508002118D3F8882022F01002C3F8882000207047D8
S3150800212803F54053D3F8882042F02002C3F88820E4
S31508002138D3F8882022F02002C3F8882000207047A8
S3150800214803F53053D3F8882042F04002C3F88820B4
S31508002158D3F8882022F04002C3F888200020704768
S3150800216803F52053D3F8882042F08002C3F8882064
S31508002178D3F8882022F08002C3F888200020704708
S3150800218803F51053D3F8882042F48072C3F88820E0
S31508002198D3F8882022F48072C3F888200020704774
S315080021A803F50053D3F8882042F40072C3F8882050
S315080021B8D3F8882022F40072C3F8882000207047D4
S315080021C803F5E053D3F8882042F48062C3F88820E0
S315080021D8D3F8882022F48062C3F888200020704744
S315080021E8000002580004025800080258000C025859
S315080021F8001002580014025800180258001C025809
S31508002208002002580024025800280258F0B40C6826
S3150800221894FAA4F4B4FA84F42BE08E68826803FB73
S3150800222803F505EB450722EA070205FB06F52A43E7
S3150800223882600E68CD68426822EA060205FB06F542
S315080022482A4342600F69C66803FB03F505EB450296
S31508002258D243164005FB07F73E43C6604E68022E72
S3150800226814D04B680668324005FB03F31343036032
S3150800227801340B6833FA04F22BD00122A24013402A
S31508002288F6D04A68013A012ADCD8C6E7FF2B0ED8E9
S31508002298066A05FB03F707FB03F3C3EB031726EAEE
S315080022A807074E6903FB06F33B430362D9E7466A09
S315080022B81B0A03FB03F707FB03F707FB03F3C3EB49
S315080022C8031726EA07074E6903FB06F33B434362EF
S315080022D8C7E70020F0BC70472DE9F04782B0D0F870
S315080022E80080CA00521A930003445A6D1B6D9A421D
S315080022F855D8C1469B1AC1EBC104A2000244526CC8
S315080023089A4200D31A460C46074602F1030A4FEAD0
S315080023189A0A15E006F1030A4FEA9A0AE3001B1B14
S315080023289D003D44A96C3B7C0093B3B2E2B240469B
S31508002338FFF704FBAB6C3344AB646B6D1E446E65E8
S3150800234809EB441303F510639B699BB2534512D3F3
S31508002358E3001B1B9A003A44516D136D99420AD241
S315080023684BB15B1AC4EBC4018A003A44566C9E42C8
S31508002378D0D31E46CEE7E3001B1B980007443A6DE8
S315080023887B6D9A420FD804F00F040123A340D8F8AE
S31508002398344824EA0304C8F83448002000E0012039
S315080023A802B0BDE8F0870020FAE77047F0B58BB0B1
S315080023B8002800F091800446056890F8BD3323B3D9
S315080023C8032384F8BD33EB6B13F4807F01D1002314
S315080023D823612068FFF778F8254655F8107B6E467E
S315080023E80FCD0FC60FCD0FC695E8030086E8030084
S315080023F8231D0ECB3846FEF7A5FF58B1022384F8ED
S31508002408BD33012528460BB0F0BD80F8BC33FFF76D
S31508002418CCFFD5E700212068FFF75CF8002365683C
S31508002428AB4216D2D900C81A82002244012082F883
S315080024383D0082F83C30A2F84230002082F83F007E
S3150800244850649064CA1A9100214408650133DBB2C6
S31508002458E5E700239D4216D9D800C11A8A00224406
S31508002468002182F8FD1182F8FC3182F8FF11C2F8C2
S315080024780412C2F80812C21A90002044C0F81012B2
S315080024880133DBB2E6E7254655F8107B6E460FCDD5
S315080024980FC60FCD0FC695E8030086E80300231D6F
S315080024A80ECB3846FFF75CF8054660B9002384F872
S315080024B83830012384F8BD33636A012B08D02068B5
S315080024C8FFF709FC9EE7022384F8BD33012599E73F
S315080024D82046FEF745FCF2E7012593E770470268B0
S315080024E890F8BC33012B19D010B5012380F8BC33FA
S315080024F8836A012B0AD004460068FFF7E0FB2068C8
S31508002508FEF7DCFF002084F8BC0310BD8369012BA5
S31508002518F1D0936B43F480339363ECE7022070475A
S3150800252838B590F8BC33012B18D00446012380F837
S31508002538BC330068FEF7C8FF2068FFF78CFB054622
S3150800254828B1002384F8BC330125284638BD2068FD
S31508002558FFF7C1FB002384F8BC33F6E70225F4E746
S3150800256868B110B50446032380F8BD33FFF7D8FFD2
S315080025782046FFF7B3FF002084F8BD0310BD0120ED
S315080025887047000070B504460D460068066C00EBF7
S31508002598411303F530639A682169012911D037492F
S315080025A88E4254D03DB9C5EBC50293002344D3F8EF
S315080025B81032002B5CD0E9B22046FDF750FF002008
S315080025C870BD12F0080F09D02D498E42F7D912F4BA
S315080025D8004FF4D04FF400429A60F0E712F0200F4B
S315080025E802D020229A60EAE712F0280FE7D1244998
S315080025F88E4206D912F4004F03D04FF400429A606F
S31508002608DDE7E900491B8A002244D2F804121B694F
S31508002618C3F31203C91AC2F81412D2F80412D2F86C
S3150800262808320B44C2F8083235B9C5EBC50293001F
S315080026382344D3F8103223B1E9B22046FDF70FFF39
S31508002648BDE704F571720121FFF796FBF4E712F46A
S31508002658004F03D04FF400429A60B0E712F0200FFB
S3150800266801D020229A60E9B22046FDF7F8FEA6E7CF
S3150800267804F571720021FFF77FFB9CE70A31544F76
S315080026880A30544F38B5044603681D6C03EB4111EC
S31508002698D1F8082B0E4B9D4207D901F5306112F483
S315080026A8004F02D04FF400438B602046FDF7CFFE5B
S315080026B8074B9D4202D92369012B01D0002038BD5A
S315080026C804F5717201212068FFF756FBF6E700BF8B
S315080026D80A30544F2DE9F84F044605682846FFF78F
S315080026E837FB08B1BDE8F88F2F4606462068FFF77E
S315080026F8FEFA0028F6D02068FFF7F9FA10F0020F5C
S3150800270804D02268536903F0020353612068FFF76F
S31508002718EEFA10F0100F15D02268936923F010030B
S315080027289361D5F8208008F00F09C8F34343022BB4
S3150800273800F08580062B00F0A5802268936943F08F
S31508002748100393612068FFF7D2FA10F4002F40F0BF
S31508002758AD802068FFF7CBFA10F4802F40F0F1809F
S315080027682068FFF7C4FA0028C0F25F812068FFF7DF
S31508002778BEFA10F4006F0AD0D5F8083813F0010F1E
S3150800278840F06D812268536903F400635361206839
S31508002798FFF7ADFA10F0006F15D02268536903F0F9
S315080027A80063536194F8F433002B40F05C810121EF
S315080027B884F8F41323685B6DC3F38303C4F8F8330A
S315080027C82046FEF7E1FA2068FFF791FA10F4805FD1
S315080027D840F04D812068FFF78AFA10F4005F40F050
S315080027E8AB812068FFF783FA10F0080F40F0BC8128
S315080027F82068FFF77CFA10F4801F40F0BE81206835
S31508002808FFF775FA10F4001F40F0C1812068FFF73A
S315080028186EFA10F0804F40F0C4812068FFF767FA17
S3150800282810F0040F3FF45EAF23685D6815F0040FD7
S3150800283840F0C081226853682B43536052E747F635
S31508002848F07318EA030F3FF478AF4FEA18184FEAFF
S31508002858C90BABEB09034FEA830AA244C8F30A0279
S31508002868DAF808122846FFF787F9C8F30A08DAF8E3
S3150800287808324344CAF80832DAF814324344CAF824
S3150800288814325AE7082204F571712846FFF774F9D5
S31508002898C8F30A184FEAC903A3EB09018A002244B8
S315080028A8D2F814324344C2F8143246E72068FFF7D0
S315080028B822FA8046B14617E007EB49130122C3F806
S315080028C8082B49462046FFF75DFE1DE007EB49132E
S315080028D80822C3F8082B49462046FFF7D3FE16E018
S315080028E809F101094FEA5808B8F1000F3FF431AF6A
S315080028F818F0010FF4D05FFA89F12068FFF70BFA90
S31508002908824610F0010FD7D11AF0080FDED11AF057
S31508002918100F04D007EB49131022C3F8082B1AF036
S31508002928200F04D007EB49132022C3F8082B1AF402
S31508002938005FD5D007EB49134FF40052C3F8082BAC
S31508002948CEE72068FFF7DFF98046B1462AE0594600
S315080029582046FDF790FD1AF0080F04D007EB491337
S315080029680822C3F808291AF0100F04D007EB4913F0
S315080029781022C3F808291AF0400F04D007EB4913A8
S315080029884022C3F808291AF0020F04D007EB4913A6
S315080029980222C3F808291AF0800F41D109F1010962
S315080029A84FEA5808B8F1000F3FF4DAAE18F0010FED
S315080029B8F4D05FFA89FB59462068FFF7B5F98246CD
S315080029C810F0010FC7D009F00F03012101FA03F22D
S315080029D8D7F8343823EA0203C7F8343807EB49131B
S315080029E8C3F8081923698B42B1D14FEAC902A2EB89
S315080029F8090293002344596C9A6C0A449A64B9F1FB
S31508002A08000FA4D1C9EBC902930023441B6D002B00
S31508002A189DD104F5717201212068FFF7ADF996E793
S31508002A2849462046FFF758FCB8E7D5F8043823F096
S31508002A380103C5F8043894F8F433012B08D0204666
S31508002A48FDF75EFD2268536903F0004353618DE67E
S31508002A58002184F8F4132046FEF796F9F2E7204693
S31508002A68FDF734FD8EE62046FDF730FDABE605F5A5
S31508002A780068D8F8043023F00103C8F80430102198
S31508002A882068FEF73FFD20E007EB46134FF67F3137
S31508002A98C3F80819D3F8002922F40012C3F8002944
S31508002AA8D3F8002942F00062C3F80029C3F8081BC6
S31508002AB8D3F8002B22F40012C3F8002BD3F8002B06
S31508002AC842F00062C3F8002B01366368B342DBD8CC
S31508002AD8D8F81C3043F00113C8F81C30236BEBB147
S31508002AE8D8F8843043F00B03C8F88430D8F8443053
S31508002AF843F00B03C8F84430D5F8003823F4FE63CE
S31508002B08C5F8003804F57172217C2068FFF734F996
S31508002B182268536903F4805353615BE6D8F8142096
S31508002B2842F22B031343C8F81430D8F8103043F090
S31508002B380B03C8F81030DFE72068FFF70DF920689F
S31508002B48FEF7D0FDE0602568FEF7BCFB227B014650
S31508002B582846FEF73DFC2046FDF79EFC2268536989
S31508002B6803F4005353613CE62046FDF78FFC2268C0
S31508002B78536903F0080353613AE600212046FDF736
S31508002B88CEFC2268536903F48013536137E60021A3
S31508002B982046FDF7BEFC2268536903F40013536107
S31508002BA834E62046FDF7C1FC2268536903F08043E2
S31508002BB8536132E62046FDF7C2FC3BE6026890F808
S31508002BC8BC33012B16D010B5012380F8BC33836AB1
S31508002BD8012B07D004460068FFF771F8002084F82F
S31508002BE8BC0310BD8369012BF4D0936B43F480337F
S31508002BF89363EFE70220704790F8BC33012B0BD09C
S31508002C0810B50446012380F8BC330068FFF763F85B
S31508002C18002084F8BC0310BD0220704790F8BC3326
S31508002C28012B0DD010B50446012380F8BC3380F873
S31508002C3838100068FFF733F8002084F8BC0310BD85
S31508002C4802207047F8B511F0800F27D101F00F055B
S31508002C58EE00771BBC00274604F5FC7404440434CC
S31508002C680744002587F8FD5101F00F012170A2607D
S31508002C78E370627802B1E180022B1ED090F8BC336B
S31508002C88012B1DD00546012380F8BC332146006870
S31508002C98FEF738FD002085F8BC03F8BD01F00F06DD
S31508002CA8F500AF1BBC0027463834044404343E46B6
S31508002CB80644012586F83D50D6E700232371DDE74B
S31508002CC80220EAE738B511F0800F20D101F00F0489
S31508002CD8E200151BAB001D4603F5FC7303440433D9
S31508002CE80544002285F8FD2101F00F01197090F8B6
S31508002CF8BC23012A1AD00446012280F8BC231946A7
S31508002D080068FEF747FD002084F8BC0338BD01F0CB
S31508002D180F04E200151BAB001D4638330344043381
S31508002D282C460444012284F83D20DDE70220EDE71D
S31508002D3870B501F00F05EE00711B8C0004F5FC74E4
S31508002D480444211D761BB4000444C4F80822C4F8B8
S31508002D5810320023C4F8143284F8FD3184F8FC5183
S31508002D680369012B06D065B9DAB20068FEF75AFD81
S31508002D78002070BDC5EBC506B4000444C4F80C228F
S31508002D88F1E7DAB20068FEF7EDFDF1E701F00F01A9
S31508002D98C1EBC1018B001844D0F81402704770B50E
S31508002DA801F00F05EE00711B8C0038340444211D10
S31508002DB8761BB4000444A2642365002363650123D3
S31508002DC884F83D3084F83C500369012B06D05DB978
S31508002DD8DAB20068FEF726FD002070BDC5EBC50609
S31508002DE8B4000444E264F2E7DAB20068FEF7BAFD12
S31508002DF8F2E738B501F00F0543689D4236D811F059
S31508002E08800F20D1CA00541AA3001C4603F5FC7388
S31508002E180344043322460244002182F8FD110122A4
S31508002E289A701D7090F8BC23012A21D00446012205
S31508002E3880F8BC2319460068FEF7B2FE7DB100206B
S31508002E4884F8BC0338BDEA00511B8B001946383391
S31508002E58034404330144012281F83D20DFE704F5E1
S31508002E687172217C2068FEF787FFE8E70120E9E709
S31508002E780220E7E710B501F00F0443689C422CD8F6
S31508002E8811F0800F1DD1E3001A1B91000A4601F5BF
S31508002E98FC71014404310244002382F8FD31002301
S31508002EA88B700C7090F8BC33012B18D0044601239C
S31508002EB880F8BC330068FEF7A0FE002084F8BC033F
S31508002EC810BDE3001A1B91000A4638310144043143
S31508002ED80244012382F83D30E1E70120F0E70220A9
S31508002EE8EEE7000030B4446B0268D2F88410704BE1
S31508002EF8194041EA8401C2F884100268D2F884109D
S31508002F0821F47F01856B41EA0541C2F88410826B7A
S31508002F1822440468D4F88810194041EA8201C4F8A2
S31508002F2888100468D4F8881021F4FE01C56B41EAB4
S31508002F380541C4F88810C16B02EB41020468D4F84D
S31508002F48A010194041EA8201C4F8A0100468D4F810
S31508002F58A01021F4FE01056C41EA0541C4F8A01049
S31508002F68046C416C01FB04240268D2F8B0101940BD
S31508002F7841EA8401C2F8B0100268D2F8B01021F408
S31508002F88FE01856C41EA0541C2F8B010826CC16C35
S31508002F9801FB02440268D2F8AC10194041EA8401E0
S31508002FA8C2F8AC10026D416D01FB02420468D4F800
S31508002FB8F010194041EA8201C4F8F0100468D4F800
S31508002FC8F01021F47C11856D41EA0541C4F8F0102A
S31508002FD8816D02EB41020468D4F8C0100B4043EA3D
S31508002FE88202C4F8C0200268D2F8C03023F47C13E1
S31508002FF8C16D43EA0143C2F8C0300268D2F8C0304E
S3150800300823F07C53016E43EA0163C2F8C030436B70
S31508003018284A1A449200C266836B02EB8303036745
S31508003028C16B03EBC1034367046C416C01FB04F1F4
S3150800303803EB81038367846CC16C01FB04F103EB22
S315080030488103C367046D416D01FB04F103EB81033A
S31508003058C0F88030816D03EBC103C0F88430C46DB5
S31508003068856E05FB04F403EB8403C0F88830016E0B
S3150800307801FB05F103EB8103C0F890300E498B423A
S3150800308807D8D0F8903093420ED9002342F8043B6B
S31508003098F7E7D0F89C3043F02003C0F89C300323A8
S315080030A880F89830012000E0002030BC704700BF47
S315080030B80300FFFF002B0010FCD30040F0B44C6857
S315080030C8002C2FD10E698C6826430C6846EA84467C
S315080030D80D6ACC6944EA05648D692C434D692C430D
S315080030E8CD682C43D0F88470806E03FB00F307EB99
S315080030F8830547F823606C6008350020CB890E4C99
S31508003108E35C834216D91418E678A3781B0443EAC5
S315080031180663647843EA0423145C234345F8043BAE
S315080031280430EBE70C698E6826430C68264346F09C
S315080031388046CDE7F0BC7047885D000870470000F8
S3150800314830B595B004464C22A04901A802F091FD75
S31508003158002C00F0388123689D4A934220D094F8C1
S3150800316898300BB32268936923F01003936102F031
S3150800317877FD054623689A6912F0080F1AD002F0F7
S315080031886FFD401B0A28F5D9D4F89C3043F0010393
S31508003198C4F89C30032384F89830012015B030BD54
S315080031A803F580736360DAE784F899302046FFF7F9
S315080031B8C5FFD7E79A6942F001029A6102F050FD05
S315080031C8054623689A6912F0010F0FD102F048FDE7
S315080031D8401B0A28F5D9D4F89C3043F00103C4F8F3
S315080031E89C30032384F898300120D7E79A6942F07F
S315080031F802029A61237C012B40D02268936943F026
S3150800320840039361637C012B3ED02268936923F4BB
S3150800321880439361A37C012B3CD02268936943F4CD
S31508003228805393612268936923F44073A1680B431A
S3150800323893612268936923F0A4039361226813694A
S3150800324823F010031361E368012B29D0002B2CD037
S31508003258022B00F09B802268936943F080039361F0
S315080032682268136943F010031361E368032B1CD122
S315080032782268936943F02003936116E022689369EC
S3150800328823F040039361BDE72268936943F48043BA
S315080032989361BFE72268936923F480539361C1E772
S315080032A82268936943F004039361A3695A1EE36984
S315080032B8013B1B0243EA4263226A013A13436269E5
S315080032C8013A216843EA0243CB61A368B3F5407F14
S315080032D862D0236E33B12268D2F8C030616E0B43D0
S315080032E8C2F8C030E36D226ED3420DD02168D1F8FA
S315080032F8C83023F00703A26E14A800EB820252F81E
S315080033084C2C1343C1F8C830236C6BB12168D1F82B
S31508003318BC3023F00703626C14A800EB820252F84B
S315080033284C2C1343C1F8BC30A36C73B12168D1F88F
S31508003338BC3023F07003E26C14A800EB820252F842
S315080033484C2C43EA0213C1F8BC30236D73B12168CB
S31508003358D1F8BC3023F4E063626D14A800EB82024E
S3150800336852F84C2C43EA0223C1F8BC302268184BA1
S315080033789A4222D00023C4F89430C4F89C3001231A
S3150800338884F898302046FFF7ADFD07E72268936969
S3150800339843F02003936188E7A36A013BE26A013A8E
S315080033A843EA0223226B013A43EA0213626A013AA4
S315080033B8216843EA0243CB608BE76268936823F087
S315080033C803039360D6E70120E8E600BFB05C00086F
S315080033D800A0004090F89830013BDBB2012B07D9D2
S315080033E8D0F89C3043F00203C0F89C30012070479F
S315080033F8CB680A68D2B9072B0ED08A68DB0643EA77
S3150800340882730A6943EA02434A691343C26E4968E2
S3150800341842F82130002070470A69CB691B0243EA43
S3150800342802438A69134343F06053EFE710B40A6905
S3150800343842EA4372072B0ED08C684B6943EA8473B9
S31508003448006F496800EBC10440F83120636000202A
S315080034585DF8044B70478B69F2E790F89830DBB251
S31508003468012B07D0D0F89C3043F00403C0F89C30F1
S3150800347801207047022380F898300268936923F080
S31508003488010393610023C0F89C301846704770B54D
S3150800349890F89840013CE4B2012C26D893FAA3F593
S315080034A8B5FA85F50668D6F8C040C4F30544A542BA
S315080034B80BD2D6F8CC401C420FD0D0F89C3043F03B
S315080034C84003C0F89C30012016E0D0F89C3043F041
S315080034D82003C0F89C3001200EE093FAA3F3B3FA50
S315080034E883F3FFF7EBFD002006E0D0F89C3043F0A5
S315080034F80203C0F89C30012070BD90F89830DBB202
S31508003508022B07D0D0F89C3043F00803C0F89C304B
S31508003518012070470368C3F8D010002070470000E0
S31508003528F0B490F89840E4B2022C40F0BA804029EA
S315080035380CD0412930D0046D8C4253D8D0F89C3031
S3150800354843F02003C0F89C300120B1E00468D4F8A1
S31508003558A05015F4FE0F0CD0D4F8A45015F07F0F20
S315080035680FD1D0F89C3043F48073C0F89C30012002
S315080035789EE0D0F89C3043F02003C0F89C30012028
S3150800358896E0D4F8A440C4F3052C446F456C0CFBAC
S3150800359805F504EB85042DE00468D4F8B05015F455
S315080035A8FE0F0CD0D4F8B45015F07F0F0FD1D0F811
S315080035B89C3043F48073C0F89C30012078E0D0F83A
S315080035C89C3043F02003C0F89C30012070E0D4F802
S315080035D8B440C4F3052C846FC56C0CFB05F504EBE5
S315080035E8850407E0C46F456D01FB05F504EB850402
S315080035F84FF0000C256805F080455560002D2CD144
S315080036082568C5F38A451560256805F0005595604F
S31508003618256805F000451561A588D561656805F42E
S315080036287025D560656805F480155561656805F4E3
S3150800363800159561E57905F07F0515626568ED0F52
S31508003648556204F108050024D6891A4FBE5DA642BC
S3150800365808D92E5D1E550134F6E7256825F060451C
S315080036681560D1E740290AD041290DD01F290FD85E
S315080036780268012303FA01F1C2F8981002E0036808
S31508003688C3F8A8C0002013E00368C3F8B8C0F9E770
S3150800369801F01F010268012303FA01F1C2F89C1020
S315080036A8F0E7D0F89C3043F00803C0F89C300120B6
S315080036B8F0BC7047885D00080368D3F89820D3F8EB
S315080036C89C001F2903D8CA4012F0010F17D01F29DA
S315080036D805D901F01F02D04010F0010F11D01F299B
S315080036E805D8012000FA01F1C3F89810704701F0CF
S315080036F81F01012000FA01F1C3F89C107047002049
S315080037087047002070470368D3F8CC300B4201D0C5
S315080037180120704700207047204A136843F00103C8
S3150800372813601E4B1B6813F0040FFAD01B4B0022BC
S315080037381A6119681A4A0A401A60184B1B6813F066
S31508003748007FFAD1154B1B6813F0006FFAD1134B9B
S315080037581B6813F0005FFAD1104B00229A61DA61F0
S315080037681A62104999621049D962104919635A634D
S315080037789963DA6319645A64196821F4802119600F
S315080037881A66996E40F2FF720A439A66D3F8D020F1
S3150800379842F48032C3F8D020704700BF004402586C
S315080037A845EDF6EA000202020000FF018002010167
S315080037B807EE900AF8EE676A07EE901AF8EE677A47
S315080037C886EEA77A07EE902AF8EE677A06EE903A1A
S315080037D8F8EE666A9FED096A66EE866A77EEA67A55
S315080037E827EE277ADDED007AF8EE677AC7EE276ABC
S315080037F8FCEEE67A17EE900A704700BF000000391B
S315080038082DE9F04182B03E4B9B6A03F00303012B76
S3150800381824D0BBB1022B28D00027002303604360BD
S315080038288360374B9E6AC6F305161A6BC2F30802FD
S31508003838551CDB6A13F0010F24D0314B5B6BC3F3BD
S31508003848CC0821E02E4B1B6813F0040F14D02C4B20
S315080038581B68C3F3C1032B4FDF40DEE7284B1B6801
S3150800386813F4807F0AD10027D7E7254B1B6813F482
S31508003878003F05D10027D0E70027CEE7224FCCE73F
S31508003888224FCAE74FF00008002E36D004461C4BD4
S31508003898DB6A13F4803F0CD0194B1B6BC3F3462322
S315080038A80133009343462A4631463846FFF780FFD8
S315080038B82060134BDB6A13F4003F0CD0104B1B6BCC
S315080038C8C3F306430133009343462A46314638462E
S315080038D8FFF76EFF60600A4BDB6A13F4802F0CD083
S315080038E8074B1B6BC3F306630133009343462A460B
S315080038F831463846FFF75CFFA06002B0BDE8F081A4
S31508003908004402580090D00300093D0000127A00CE
S315080039182DE9F04182B03E4B9B6A03F00303012B65
S3150800392824D0BBB1022B28D00027002303604360AC
S315080039388360374B9E6AC6F305369A6BC2F308024C
S31508003948551CDB6A13F0100F24D0314BDB6BC3F31D
S31508003958CC0821E02E4B1B6813F0040F14D02C4B0F
S315080039681B68C3F3C1032B4FDF40DEE7284B1B68F0
S3150800397813F4807F0AD10027D7E7254B1B6813F471
S31508003988003F05D10027D0E70027CEE7224FCCE72E
S31508003998224FCAE74FF00008002E36D004461C4BC3
S315080039A8DB6A13F4002F0CD0194B9B6BC3F3462321
S315080039B80133009343462A4631463846FFF7F8FE50
S315080039C82060134BDB6A13F4801F0CD0104B9B6BDB
S315080039D8C3F306430133009343462A46314638461D
S315080039E8FFF7E6FE60600A4BDB6A13F4001F0CD08B
S315080039F8074B9B6BC3F306630133009343462A467A
S31508003A0831463846FFF7D4FEA06002B0BDE8F0811B
S31508003A18004402580090D00300093D0000127A00BD
S31508003A282DE9F04182B0424B9B6A03F00303012B50
S31508003A3824D0BBB1022B28D000250023036043609D
S31508003A4883603B4B9C6AC4F305541A6CC2F308029C
S31508003A58561CDB6A13F4807F24D0354B5F6CC7F39A
S31508003A68CC0720E0324B1B6813F0040F14D0304BF8
S31508003A781B68C3F3C1032F4DDD40DEE72C4B1B68DB
S31508003A8813F4807F0AD10025D7E7294B1B6813F45E
S31508003A98003F05D10025D0E70025CEE7264DCCE71F
S31508003AA8264DCAE700272B1C18BF0123002C08BF80
S31508003AB80023002B39D080461D4BDB6A13F4800F90
S31508003AC80DD01B4B1B6CC3F34623013300933B46AF
S31508003AD8324621462846FFF76BFEC8F80000144B05
S31508003AE8DB6A13F4000F0DD0114B1B6CC3F30643A6
S31508003AF8013300933B46324621462846FFF758FECF
S31508003B08C8F804000A4BDB6A13F0807F0DD0084B0F
S31508003B181B6CC3F30663013300933B4632462146C2
S31508003B282846FFF745FEC8F8080002B0BDE8F08148
S31508003B38004402580090D00300093D0000127A009C
S31508003B48154B1B6903F03803182B0ED8DFE803F06A
S31508003B580F0D0D0D0D0D0D0D210D0D0D0D0D0D0D69
S31508003B68160D0D0D0D0D0D0D1800002070470A4B8A
S31508003B781B68C3F3C1030948D8407047084870470B
S31508003B8800B585B001A8FFF73BFE019805B05DF8BA
S31508003B9804FB0448704700BF004402580090D0034D
S31508003BA800127A0000093D00044B9B6903F00F03D5
S31508003BB8034AD35C03F01F03D840704700440258F1
S31508003BC8985D0008044BDB69C3F30213034AD35C08
S31508003BD803F01F03D840704700440258985D000850
S31508003BE8044BDB69C3F30223034AD35C03F01F03C0
S31508003BF8D840704700440258985D000800B585B05B
S31508003C08C2B24F4BD358020EC0F304218A40134060
S31508003C18CB4040EA03404B4B984228D033D8A3F50B
S31508003C288133A3F58073984266D019D8A3F58033F3
S31508003C38984251D003F5407398420FD1FFF780FF99
S31508003C48414B9B69C3F30323404AD35C03F01F0324
S31508003C58D840FFF7A9FFFFF7C3FF24E0002022E0BA
S31508003C683B4B984248D003F57D43984209D1364BD9
S31508003C781B6813F0005F59D001A8FFF7D1FE029818
S31508003C8811E000200FE0334B98423FD00ED9324B53
S31508003C98984242D003F5407398423ED0A3F5803344
S31508003CA8984233D0002005B05DF804FBA3F58033AD
S31508003CB8984203D003F5407398420BD1224B1B68F0
S31508003CC813F0040F34D0204B1B68C3F3C1032348F1
S31508003CD8D840E8E70020E6E7FFF732FF1A4B9B696A
S31508003CE8C3F30323194AD35C03F01F03D840FFF72D
S31508003CF85BFFFFF767FFD6E7134B1B6813F0006FE8
S31508003D0812D001A8FFF704FE0298CCE70E4B1B68F1
S31508003D1813F4807F0ED10020C5E70B4B1B6F13F0F9
S31508003D28020F09D10020BEE70020BCE70020BAE749
S31508003D380020B8E70A48B6E74FF40040B3E700BFE3
S31508003D484C4402580803020700440258985D0008C4
S31508003D580803010708000407080005070090D003B0
S31508003D6800093D0001F00303032B24D011F0010FCD
S31508003D780BD01D4BDA6822F03002DA60DA680243A3
S31508003D88DA60DA6842F08802DA6011F0020F11D0B8
S31508003D98154BD3F80C2122F03002C3F80C21D3F8BE
S31508003DA80C211043C3F80C01D3F80C2142F0880201
S31508003DB8C3F80C2170470C4BDA6822F03002DA6037
S31508003DC8D3F80C2122F03002C3F80C21DA68024332
S31508003DD8DA60D3F80C211043C3F80C019A6942F04B
S31508003DE810029A61704700BF0020005230B411F0E3
S31508003DF8010F0BD0104DEB6823F4E663EB60EC6813
S31508003E0842EA00231C4344F08404EC6011F0020FD4
S31508003E180FD00949D1F80C3123F4E663C1F80C31FF
S31508003E28D1F80C3142EA0022134343F08403C1F85F
S31508003E380C3130BC704700BF00200052F8B5474B1C
S31508003E481B7D012B00F088800F460446434B012250
S31508003E581A7500229A61436813F0010F0DD10026DE
S31508003E68636813F0020F12D1CEB92368012B1BD051
S31508003E784FF0FF333B60A56859E001214CF25030FA
S31508003E88FDF7F6FF06460028EAD00126E8E70221EC
S31508003E984CF25030FDF7ECFF0028E5D001262F4BF1
S31508003EA800221A753046F8BD61682069FFF75AFF7F
S31508003EB8636813F0010F12D1636813F0020FEED08E
S31508003EC802214CF25030FDF7D3FF00B10126244AEF
S31508003ED8D2F80C3123F00803C2F80C31DFE70121C8
S31508003EE84CF25030FDF7C4FF00B101261C4AD368CE
S31508003EF823F00803D360DFE701214CF25030FDF7C1
S31508003F08B7FF0646164AD168164B0B40D3601CE025
S31508003F1802214CF25030FDF7ABFF0646104AD2F89C
S31508003F280C11104B0B40C2F80C319EB90135E368E9
S31508003F38A2681344AB42B2D9226961682846FFF7DA
S31508003F4855FF636813F0010FD6D1636813F0020FA3
S31508003F58EBD0DDE73D60A2E70226A3E718190020A3
S31508003F6800200052FBF8FFFF184AD2F8883043F4BD
S31508003F787003C2F88830164B1A6842F001021A60B4
S31508003F8800221A6118681349014019609A61DA61B2
S31508003F981A629A62DA621A635A639A63DA631A6465
S31508003FA85A64196821F4802119601A660A4B1A6836
S31508003FB80A4B1340B3F1005F02D2094B01221A607B
S31508003FC8024B4FF000629A60704700BF00ED00E0B0
S31508003FD8004402587FEDF6EA0010005C0000FFFF77
S31508003FE80881005198B108B50346D0F8B40210B153
S31508003FF80020C3F8B40209B1C3F8B0121846012361
S3150800400880F89C320270FCF7A5FA002008BD022049
S31508004018704710B50446012380F89C32D0F8B432AC
S315080040285B68017998472046FCF709FB2046FCF7A8
S31508004038F6FA002010BD19B1C0F8B412002070476E
S315080040480220704708B5FCF7F2FA002008BD08B543
S31508004058D0F8B43233B11B68984708B9002008BDB0
S315080040680220FCE70220FAE708B5D0F8B4325B6804
S315080040789847002008BD38B5044600F52A7528462D
S3150800408800F04EF90123C4F89432B4F8AE32C4F8F5
S31508004098983294F8A81201F01F03012B0FD05AB2D0
S315080040A83AB1022B10D001F080012046FCF7E2FA5B
S315080040B803E02946204600F0E1FA002038BD2946E3
S315080040C8204600F00FFBF8E72946204600F03AFBA1
S315080040D8F3E738B50446A9BB1046D4F89432032B3F
S315080040E803D0052B25D0002038E0D4F86031D4F861
S315080040F8642193420DD99B1AC4F860319A4206D9AD
S315080041089AB20146204600F06EFC002026E092B2DC
S31508004118F7E7D4F8B4321B691BB194F89C22032A32
S3150800412804D0204600F067FC002017E02046984790
S31508004138F7E70025C4F8945229462046FCF79AFA68
S3150800414828460BE00A46D0F8B4329B693BB190F88A
S315080041589C12032905D111469847002038BD02202C
S31508004168FCE70220FAE710B50446002956D110469E
S31508004178D4F89432022B09D0002B18BF042B44D04C
S3150800418894F8A032012B45D0002010BD236A626A34
S3150800419893421BD8E169B1FBF2F302FB13132BB95F
S315080041A88A4203D8D4F8983299421DD3D4F8B4323F
S315080041B8DB681BB194F89C22032A23D08021204669
S315080041C8FCF758FA204600F021FCD9E79A1A226229
S315080041D892B20146204600F0FEFB00231A4619460D
S315080041E82046FCF767FACBE700221146204600F07E
S315080041F8F2FB0021C4F898120B460A462046FCF73B
S3150800420859FABDE720469847D8E780212046FCF7A3
S3150800421831FAB5E7002084F8A002B6E70A46D0F8CE
S31508004228B4325B693BB190F89C12032905D1114653
S3150800423898470020A9E70220A7E70220A5E770B556
S315080042480446402300221146FCF701FA0125C4F862
S3150800425858514026C4F86461334600228021204616
S31508004268FCF7F5F9A561666284F89C520023C4F840
S3150800427894326360C4F8A432D4F8B8322BB1D4F8AF
S31508004288B4325B68002120469847002070BD017447
S315080042980020704790F89C3280F89D32042380F8F5
S315080042A89C320020704790F89C32042B01D00020DD
S315080042B8704790F89D3280F89C32F8E708B590F870
S315080042C89C32032B01D0002008BDD0F8B432DB6934
S315080042D8002BF8D09847F6E700207047002070476B
S315080042E80020704708B5012280F89C22D0F8B4222D
S315080042F8526801799047002008BD002302781AB150
S315080043080133DBB20130F9E71846704708B54B8820
S31508004318012B00D008BDC0F8A43200F06CFBF9E701
S315080043280B7803704B7843708B78CA7803EB0223B3
S3150800433843800B794A7903EB022383808B79CA7900
S3150800434803EB0223C380704710B504468021FCF7A7
S3150800435891F900212046FCF78DF910BD30B583B0D8
S3150800436805460C460023ADF806304A88130A013B71
S31508004378062B00F2A480DFE803F004182CA2A28614
S315080043889300D0F8B0321B680DF10601007C9847F7
S31508004398BDF806201AB1E388002B40F09480E3881C
S315080043A8002B00F09A8003B030BD037C43B9D0F8DF
S315080043B8B4329B6A0DF10600984702234370E7E773
S315080043C8D0F8B432DB6A0DF1060098470223437029
S315080043D8DEE7D2B2052A52D8DFE802F003101D2A12
S315080043E83744D0F8B0325B6823B10DF10601007C7A
S315080043F89847CDE72146FFF7A7FFD4E7D0F8B032AC
S315080044089B6823B10DF10601007C9847C0E7214651
S31508004418FFF79AFFC7E7D0F8B032DB6823B10DF18A
S315080044280601007C9847B3E72146FFF78DFFBAE7F0
S31508004438D0F8B0321B6923B10DF10601007C984704
S31508004448A6E72146FFF780FFADE7D0F8B0325B69EB
S3150800445823B10DF10601007C984799E72146FFF735
S3150800446873FFA0E7D0F8B0329B6923B10DF10601B6
S31508004478007C98478CE72146FFF766FF93E72146B5
S31508004488FFF762FF8FE7037C33B9D0F8B4325B6B6A
S315080044980DF1060098477BE72146FFF755FF82E7A7
S315080044A8037C43B9D0F8B4321B6B0DF10600984764
S315080044B8072343706CE72146FFF746FF73E7214653
S315080044C8FFF742FF6FE79A4228BF1A46ADF806205B
S315080044D80146284600F072FA61E7284600F08BFA8A
S315080044E861E738B504468B88F3B9CB88E3B94B88B6
S315080044F87F2B19D803F07F0590F89C32032B0CD034
S3150800450880F89E522946FCF7C5F8204600F073FA4B
S3150800451835B1022384F89C3209E0FFF715FF06E057
S31508004528012384F89C3202E02046FFF70DFF38BDC8
S3150800453838B504460D468978284B197001290ED8CE
S3150800454890F89C32022B0ED0032B21D02946FFF770
S31508004558FBFE224B19782046FFF786FD02E029461E
S31508004568FFF7F2FE38BD81B14160032380F89C321B
S31508004578FFF76DFD022803D0204600F03CFAF1E764
S3150800458829462046FFF7E0FEECE700F034FAE9E7AB
S3150800459889B1436899421DD0D9B2FFF765FD0F4B1B
S315080045A8197861602046FFF752FD02280DD020468B
S315080045B800F021FAD6E7022380F89C324160FFF71B
S315080045C853FD204600F017FACCE729462046FFF7A0
S315080045D8BBFEC7E700F00FFAC4E700BF18050020BE
S315080045E808B5CB88012B0CD190F89C325AB29AB1EF
S315080045F8022B09D9032B0FD10122011D00F0DEF980
S3150800460801E0FFF7A1FE08BD0146002341F8083F6F
S31508004618012200F0D3F9F6E7FFF796FEF3E708B5A7
S3150800462890F89C32013B022B12D8CB88022B0CD16E
S315080046380123C360D0F8A4320BB10323C360022256
S3150800464800F10C0100F0BAF908BDFFF77DFEFBE79B
S31508004658FFF77AFEF8E708B590F89C32013B022B7B
S3150800466809D84B88012B00D008BD0023C0F8A4320E
S3150800467800F0C1F9F8E7FFF767FEF5E708B50B7824
S3150800468803F06003202B05D0402B03D043B1FFF776
S315080046985BFE03E0D0F8B4329B689847002008BD53
S315080046A84B78092B1BD8DFE803F011171A141A08D8
S315080046B8051A0E0BFFF752FEF0E7FFF712FFEDE7B4
S315080046C8FFF736FFEAE7FFF78BFFE7E7FFF7A7FFEE
S315080046D8E4E7FFF71BFEE1E7FFF7BDFFDEE7FFF7B5
S315080046E833FEDBE738B505460C460B7803F060035E
S315080046F8202B06D0402B04D01BB1FFF725FE00203F
S3150800470838BD95F89C32013B022B16D82379012B24
S315080047180ED8D5F8B4329B68214628469847E388C8
S31508004728002BECD10028EAD1284600F064F9E6E720
S3150800473821462846FFF708FEE1E721462846FFF7FF
S3150800474803FEDCE738B504468A880B7803F060036D
S31508004758202B08D0D0B2402B05D05BB12046FFF7F6
S31508004768F3FD002005E0D4F8B4329B682046984744
S31508004778002038BD202B13D04B78012B43D05DB2CF
S31508004788002D73D0032B40F0F78094F89C32022B47
S315080047980CD0032B21D02046FFF7D6FD0020E8E7EA
S315080047A8D4F8B4329B6820469847E2E7B0F180030C
S315080047B818BF0123002808BF00234BB1014620462D
S315080047C8FBF758FF80212046FBF754FF0020D0E767
S315080047D82046FFF7B9FD0020CBE74B884BB9B0F167
S315080047E8800318BF0123002808BF00230BB1CB8814
S315080047F823B1204600F0FFF80020BAE70146204614
S31508004808FBF738FFF5E794F89C32022B06D0032B02
S315080048181BD02046FFF798FD0020AAE7B0F18003D1
S3150800482818BF0123002808BF00234BB101462046BC
S31508004838FBF720FF80212046FBF71CFF002098E79E
S315080048482046FFF781FD002093E74B88002B40F0B0
S31508004858988010F07F0F04D1204600F0CCF800208D
S3150800486887E701462046FBF70DFFF5E794F89C32E3
S31508004878022B06D0032B2FD02046FFF765FD002014
S3150800488877E7B0F1800318BF0123002808BF002383
S315080048989BB912F0800F15D100F07F0000EB80005D
S315080048A8830003F5A8712144043100250D6002220E
S315080048B8204600F083F828465BE72046FFF744FDC4
S315080048C8002056E700F07F0000EB8000830003F124
S315080048D8100121440431E8E752B2002A24DB00F02B
S315080048E80F0303EB83039D002544D5F858314BB3D2
S315080048F8002A2CDB00F07F0202EB8202930003F504
S31508004908A87525440435802814BF002301230028E8
S3150800491808BF01232BB300232B6002222946204611
S3150800492800F04CF8002024E700F00F0303EB83039C
S315080049389D002544AB69002BDAD12046FFF704FD14
S31508004948002016E72046FFF7FFFC002011E700F0D5
S315080049587F0202EB8202930003F110052544043511
S31508004968D1E701462046FBF731FE10B101232B603B
S31508004978D3E700232B60D0E72046FFF7E5FC0020A5
S31508004988F7E60020F5E6C0B170B50D4616460446AA
S31508004998FFF7B3FC013040003080287003236B70A2
S315080049A80223217841B101345A1CD2B2E9540233A0
S315080049B8DBB20021A954F4E770BD704710B5134659
S315080049C80222C0F89422C36103620A460021FBF753
S315080049D869FE002010BD08B513460A460021FBF7F4
S315080049E861FE002008BD08B513460A460021FBF7F4
S315080049F861FE002008BD08B50423C0F894320023D8
S31508004A081A461946FBF74EFE002008BD08B50523C9
S31508004A18C0F8943200231A461946FBF74BFE0020C5
S31508004A2808BD0000014B00225A7070471C0500207B
S31508004A38034BFE22DA7018710222A3F84420704745
S31508004A481C05002010B5054C00232370FFF7EAFF64
S31508004A58FF23E3700123A4F8443010BD1C05002089
S31508004A68064BFF22DA7000221A71597859719A7121
S31508004A78DA711A720622A3F8442070471C0500202A
S31508004A8808B50020FFF7D4FF08BD0000074BFF2232
S31508004A98DA70074A9A6400221A715A719A710722BB
S31508004AA8C3F807200822A3F8442070471C050020ED
S31508004AB8B85D0008044BFF22DA7042689A6401223E
S31508004AC8A3F84420704700BF1C05002008B531200C
S31508004AD8FFF7AEFF08BD000038B5084CFF23E370A2
S31508004AE800252571657100F00BFAA071E57125722C
S31508004AF865720723A4F8443038BD00BF1C0500209A
S31508004B0838B5FFF78FFF0E4C01252570FF23E37094
S31508004B18102323710023637100F0F2F9A07100F0E5
S31508004B2801FAE07100F0FEF9C0F3072020726572F9
S31508004B38A5720823A4F8443000F07CFA38BD00BFF3
S31508004B481C05002038B5054600F0DAF96A7890425F
S31508004B580FD90A4CA16C201D00F098FCFF23E370BE
S31508004B686A78A36C1344A3646B780133A4F84430B9
S31508004B7838BD2220FFF75CFFFAE700BF1C050020B6
S31508004B8838B5044600F0BCF96378984211D96168CB
S31508004B980A4DA9646278281D00F078FCFF23EB709B
S31508004BA86278AB6C1344AB6463780133A5F8443078
S31508004BB838BD2220FFF73CFFFAE700BF1C05002096
S31508004BC8F8B50546174600244E1E39B115F8013BB7
S31508004BD81C44E4B200F0DCF93146F5E73C600120F4
S31508004BE8F8BD000010B5084CFF23E370E21D4168C4
S31508004BF8A06CFFF7E5FF207100236371A3710823F2
S31508004C08A4F8443010BD00BF1C05002038B5054679
S31508004C180D4B9C6C00F074F96A1C411E204600F086
S31508004C280DFA60B1084CFF23E37000F069F9013802
S31508004C38A36C0344A3640123A4F8443038BD312087
S31508004C48FFF7F6FEFAE700BF1C05002010B5044674
S31508004C5800F056F901386378984213DD114BFF22A4
S31508004C68DA700122A3F84420617879B1A21C0D4BA9
S31508004C78986C00F0E3F988B161780A4A936C0B449A
S31508004C88936410BD2220FFF7D3FEFAE700F0E6F991
S31508004C980028F6D13120FFF7CBFEF2E73120FFF7DF
S31508004CA8C7FEEEE71C05002008B54168074B986C57
S31508004CB800F0C8F930B1054BFF22DA700122A3F8D3
S31508004CC8442008BD3120FFF7B3FEFAE71C0500208B
S31508004CD808B500F0BBFB034BFF22DA700122A3F8E4
S31508004CE8442008BD1C05002008B589B200F0E6F87E
S31508004CF808BD0000054B00221A709A6483F8432001
S31508004D08A3F844209A705A70704700BF1C05002003
S31508004D18034B1B780BB1012070470020704700BF72
S31508004D281C050020024B002283F84320704700BF69
S31508004D381C05002008B50378FF2B23D0354A1278BE
S31508004D48012A2BD1C93B352B53D8DFE803F040524B
S31508004D58524F52524C43494652525252525252524A
S31508004D68525252525252525252525252525252520D
S31508004D785252525252525252312B282E52525234B1
S31508004D8852373A3DFFF7BCFE224B93F84330012BC6
S31508004D9833D0204BB3F94410002932DC08BDFFF79D
S31508004DA8D1FEF1E7FFF7ECFEEEE7FFF783FEEBE748
S31508004DB8FFF718FFE8E7FFF769FEE5E7FFF760FE84
S31508004DC8E2E7FFF74DFEDFE7FFF73CFEDCE7FFF714
S31508004DD81DFFD9E7FFF73AFFD6E7FFF77DFED3E7CA
S31508004DE8FFF762FFD0E7FFF773FFCDE7FFF76EFE21
S31508004DF8CAE72020FFF71CFEC6E71020FFF718FEB3
S31508004E08C7E71846012380F843300330FFF76CFFDD
S31508004E18C4E700BF1C05002010B5FFF76BFF00F0BC
S31508004E2885FD064C0123237000F05AFE00232370E3
S31508004E3800F0DCF90223237010BD00BFEC04002043
S31508004E4800B583B00DF10701184800F0FDFD0128EB
S31508004E5810D00DF10701154800F07AFE012812D086
S31508004E680DF10701114800F041FA012814D003B0E2
S31508004E785DF804FB0E4B01221A709DF807100B48C3
S31508004E88FFF758FFE5E70A4B00221A709DF8071046
S31508004E980648FFF74FFFE3E7054B02221A709DF80D
S31508004EA807100248FFF746FFE1E700BF680500203C
S31508004EB8EC04002008B500F0DFF908BD38B504464B
S31508004EC80D460E4B1B78012B09D00C4B1B7853B19A
S31508004ED80A4B1B78022B0BD0FFF724FF38BDC9B243
S31508004EE800F080FDF1E7E9B2204600F015FEEFE78D
S31508004EF8E9B2204600F0D0F9EEE700BFEC0400203E
S31508004F08074B1B78022B05D0032B05D0012B05D0A0
S31508004F18402070473F207047002070470820704798
S31508004F28EC040020074B1B78022B05D0032B05D071
S31508004F38012B05D0402070473F2070470020704756
S31508004F4808207047EC04002008B5FFF7E1FE034681
S31508004F5800B10123184608BD08B500F073FA00F039
S31508004F6813F800F053FE00F065F8FFF755FF00F058
S31508004F7851F808BD08B500F00BF800F05BFEFFF71E
S31508004F885FFF00F009F808BD08B5FBF7ABFD08BDDB
S31508004F9808B5FBF7ACFD08BD08B5FFF7D5FF01282E
S31508004FA803D00B4B1B78012B00D008BD00F050FE30
S31508004FB8084B1B68084A1268134403F5FA739842A3
S31508004FC8F3D3034B00221A7000F040FAEDE700BF4E
S31508004FD8AC050020A8050020B0050020014B186084
S31508004FE8704700BFA8050020014B1868704700BF26
S31508004FF8A805002008B5054B1B78012B00D008BD6D
S3150800500800F026FE024B1860F9E700BFAC05002041
S31508005018B005002008B5044B01221A70FFF7EAFF0D
S31508005028FFF7BAFF08BD00BFAC05002008B5FFF7B3
S31508005038AFFFFCE708B500F05FFB08BD08B500F050
S3150800504867FB08BD08B500F09DFB08BD08B500F06C
S31508005058E3FB08BD08B500F02DFC08BD08B500F04F
S31508005068B5FB034608B9184608BD00F001FC034617
S31508005078F9E70000094B03F11801002232B19A74C6
S3150800508800225A61064B054A1A6070479A74596194
S31508005098183318310132D2B2F0E700BFF405002000
S315080050A8240600200A4B1B6883B110B45C69084AB9
S315080050B8146019749860D86000225A741860013907
S315080050C808445860987C5DF8044B7047FF20704781
S315080050D82406002038B504460D4601281CD8620067
S315080050E82244D100114B0B445A7C1B7C9A4219D096
S315080050F80E4B0B44DA6815705A7C01325A74DA6812
S315080051080132DA605B689A420ED9084A084651584D
S315080051180244D160012038BD4FF4E1710448FFF715
S3150800512885FFDCE70020F6E70120F4E7F405002010
S31508005138C05D000808B50146024B1878FFF7CAFF94
S3150800514808BD00BF2806002038B504460D460128C4
S315080051581ED804EB4403DA00124B13445B7CEBB10C
S3150800516862002244D1000F4B0B449A6812782A70C1
S315080051785A7C013A5A749A6801329A605B689A426C
S315080051880ED9084A0846515802449160012006E09B
S315080051984FF4F2710448FFF749FFDAE7002038BDF3
S315080051A80120FCE7F4050020C05D000808B50146A3
S315080051B8024B1878FFF7C8FF08BD00BF6C06002029
S315080051C810B50446012806D804EB4404E200054B4A
S315080051D81344587C10BD4FF401710348FFF726FFA6
S315080051E8F2E700BFF4050020C05D000838B5FFF7F0
S315080051F841FF1B4C4021601CFFF754FF2070194DD6
S315080052084021681CFFF74EFF28702378FF2B1DD016
S31508005218FF281BD0144C002214492046FEF7E2FE4C
S3150800522813492046FEF707FF0120FBF764FC2046D2
S31508005238FEF708FFFCF7F6FED4F8C002FDF7BEFC39
S31508005248FFF7D2FEB0F5FA6F05D338BD85210948B0
S31508005258FFF7ECFEDEE74FF4FA60FFF7BFFEF4E768
S31508005268280600206C060020B006002090040020BE
S315080052782C040020C05D000810B5064CD4F8C002FE
S31508005288FDF7BAFC2046FEF7C4FE0020FBF733FC00
S3150800529810BD00BFB006002070B506460D463F296A
S315080052A806D82846FFF746FF012806D100240FE04E
S315080052B8BB210D48FFF7BAFEF3E7BF210A48FFF7F7
S315080052C8B5FEF3E7C8210848FFF7B0FE0134A4B2D3
S315080052D8ABB2A34207D9FFF75BFE305DFFF72AFF9B
S315080052E80128F3D0EEE770BDC05D000870B5064624
S315080052F80D461F4BD3F8C002FDF7ECF91D4B1C7879
S315080053089CB91D48FFF752FF012801D0204670BDF9
S31508005318194B1B78013BDBB23E2BF7D8154B0122FC
S315080053281A70164B00221A70F0E7144B1B780133D3
S3150800533811481844FFF73AFF0446012801D000240B
S31508005348E4E70E4B1A780132D2B21A700A4B1B7868
S315080053589A4201D00024D9E70949304600F096F860
S31508005368044B00221A70054B1B782B70CEE700BF3A
S31508005378B0060020B409002074090020B5090020E9
S315080053887509002030B583B0144B1878FFF718FF55
S3150800539808B30546402800D9402500240AE04FF4FA
S315080053A8A4710F48FFF742FE9DF807200D4B1A55C2
S315080053B80134E4B2A54208D90DF10701074B18785C
S315080053C8FFF7C2FE0128EFD0E9E7ABB2054A81210B
S315080053D80548FBF767F903B030BD00BF280600206B
S315080053E8C05D0008B4050020B006002070B5044664
S315080053F8FBF7FAFB064621460F48FBF7FEF885B287
S31508005408002406E04FF4B5710C48FFF70FFE013487
S31508005418A4B2AC4207D2315D094B1878FFF75AFE99
S315080054280128F4D0EEE7FBF7DFFB4023024601210B
S315080054380148FBF73FF970BDB0060020C05D0008BB
S315080054486C06002008B500F010FC08BD10B5FFF77B
S31508005458FDFD00B910BDFBF737FB0028FAD0FFF7AA
S3150800546829FDFBF793FC00F0C9FBFFF7F3FD054B95
S315080054780340054A9360FFF7EDFD446800F0F7FB23
S31508005488A047E7E780FFFF1F00ED00E070B50D466F
S315080054980446531E9EB23AB115F8013B04F8013B7F
S315080054A8FFF776FD3246F4E770BD000038B50546C5
S315080054B8002401E00134E4B20E2C12D8FFF768FD87
S315080054C804EB44029300084AD358AB42F2D804EBDB
S315080054D844029100044A0A4452681344AB42E9D983
S315080054E800E0FF24204638BDE85D000808B5C1F38A
S315080054F8090363B903688B4201D1012008E040F823
S31508005508041B4FF48062FFF7C1FF012000E000206A
S3150800551808BD2DE9F04107460068FFF7C7FFFF28D1
S3150800552804D14FF000084046BDE8F081FCF754FC6A
S3150800553800264FF0010805E04FF00008B8F1000F03
S315080055481DD001361F2E1AD83D68740125443C44DF
S315080055580434FFF71DFD224629460120FCF704FD01
S3150800556858B900231F2BE9D8595DC9B2E25CD2B2F3
S315080055789142E1D10133DBB2F4E74FF00008FCF7BA
S3150800558859FCD0E770B50E460E4B984212D0054620
S315080055980D4B994209D10B4C254624B1314628466C
S315080055A8FFF7A4FF58B1204670BDFFF7B2FF20B138
S315080055B82C46F2E7054C2546EFE70024EDE70024DC
S315080055C8F1E700BFBC0D002000000208B80900205A
S315080055D82DE9F84306460C4617461D46DFF884802B
S315080055E801EA08080368B3F1FF3F0AD03368434560
S315080055F80ED14FF00109B9F1010F12D04846BDE89E
S31508005608F8834146FFF772FF81460028F3D0EDE795
S3150800561841463046FFF7B6FF0646E8B14FF001099E
S31508005628E9E73368E41A3444043405E017F8013B1B
S3150800563804F8013B013DE1D0FFF7AAFC331DE31A44
S31508005648B3F5806FF2D308F580613046FFF79AFF05
S31508005658064620B1041DE9E74FF00009CEE74FF0EA
S315080056680009CBE700FCFFFF70B586B004460D4677
S3150800567800230093884203D80E2938D8012600E06B
S31508005688002616B9304606B070BDFCF7A5FB01E042
S315080056980134E4B2AC4227D8FFF77AFC154963000F
S315080056A823449A008B188A585B68002B18BFB2F1F6
S315080056B8FF3F18D000230193202305930A46630069
S315080056C81819810008461144497A02910244137A46
S315080056D8039301230493694601A8FEF7AFFB002844
S315080056E8D6D0002600E00026FCF7A4FBCAE7002669
S315080056F8C8E700BFE85D00084FF0FF33024A1360A9
S31508005708024A1360704700BFB8090020BC0D002084
S3150800571870B504460D4616464A1E154B1B1A9A427C
S3150800572803D9002001280ED070BDFFF7BFFEFF2859
S3150800573801D10020F8E728190138FFF7B7FEFF2836
S3150800574814D00120EEE70B4B23400B4A934206D0B0
S315080057582B46324621460948FFF73AFFE4E72B4627
S31508005768324621460648FFF733FFDDE70020DBE728
S31508005778FFFF1F0800FCFFFF00000208B809002009
S31508005788BC0D002070B54A1E0F4B1B1A9A4205D944
S31508005798FF210E460020012812D070BD05460C468A
S315080057A8FFF784FE064660190138FFF77FFE0146B3
S315080057B8FF2818BFFF2E01D00120ECE70020EAE7F2
S315080057C83046FFF751FFE8E7FFFF1F08104B1B6835
S315080057D8B3F1FF3F01D10120704700B583B00C4AE9
S315080057E8536891680B44D1680B4411690B44516995
S315080057F80B4491690B44D26913445B42019301AA8D
S3150800580804210448FFF784FF03B05DF804FB00BFD2
S31508005818BC0D0020980202080D4B1B680D4A126839
S315080058281A440D4B1B6813440C4A126813440C4A55
S3150800583812681A440B4B1B681A440B4B1B68134413
S315080058480A4A1268DA4201D10120704700207047D7
S315080058580000020804000208080002080C000208F2
S315080058681000020814000208180002089802020824
S3150800587808B50E4B1B68B3F1FF3F07D10C4B1B68E5
S31508005888B3F1FF3F09D10123184608BD0748FFF7BA
S3150800589840FE03460028F7D0F0E70548FFF739FE2B
S315080058A803460028F0D00123EEE700BFBC0D002010
S315080058B8B80900200048704700000208F0B4194DDE
S315080058C82C6D24F040542C65002401E00134E4B220
S315080058D8112C23D8144D15F8146005EB44056F7878
S315080058E8F51905FB00054FF4FA5CBCFBF5FC05FB4E
S315080058F80CF5B5F5FA5FE9D135463D4405FB000CCC
S315080059084FF4FA55B5FBFCF50D80013DADB2B5F57A
S31508005918007FDBD216701F70012000E00020F0BC63
S31508005928704700BF00440258C45E000870B58AB0C4
S315080059380023ADF826308DF825308DF8243009ABCC
S315080059480DF125020DF126014FF4FA70FFF7B6FF9F
S3150800595800283CD0204C214B23600025A560E56033
S31508005968012626746574A574BDF826306361A66198
S315080059789DF82530E3619DF8243023626662A662A5
S31508005988E66226636563A663E563256404236364A0
S31508005998A564E36426656365A565E66525666566A3
S315080059A8A3662046FDF7CCFB0195029503960723C7
S315080059B8049340F2676305930693079501A9204661
S315080059C8FDF708FD2046FDF748FD0AB070BDB82169
S315080059D80348FFF72BFBBDE7C011002000A00040D5
S315080059E89C5E000810B58AB040F2E1730193002363
S315080059F8029303930904049105930693079308935E
S31508005A08522309930123024601A90E48FDF73FFDD3
S31508005A1808B10AB010BD01210A48FDF76EFD002835
S31508005A28F7D100F015F900F1320401210548FDF710
S31508005A386AFE0028EDD0FFF7ABFA00F009F9A04294
S31508005A48F3D9E6E7C011002030B58BB004460D46F9
S31508005A5800211048FDF730FE10B900200BB030BD04
S31508005A6823466A4600210B48FDF75AFD68B9009A8D
S31508005A7840F267639A4201D00020EFE7019B33B9E9
S31508005A889DF80E302B700120E8E70020E6E7002095
S31508005A98E4E700BFC0110020054BDB6913F0200FAF
S31508005AA804D0034B5B6A03700120704700207047D7
S31508005AB80048004010B5094B986200F0C9F800F193
S31508005AC80A04064BDB6913F0800F05D1FFF760FA65
S31508005AD800F0BEF8A042F4D910BD00BF0048004047
S31508005AE810B588B0002300934FF4614201920293DF
S31508005AF8039304930C22059206930793054C69466B
S31508005B082046FBF737FA236843F00103236008B0F9
S31508005B1810BD00BF0048004070B506460D4640292E
S31508005B280ED82846FFF7C6FF0024ABB2A3420CD905
S31508005B38FFF72EFA305DFFF7BDFF0134A4B2F4E78C
S31508005B4882210248FFF772FAEBE770BDE85E0008A3
S31508005B5870B5254B1C78BCB92448FFF79DFF01286A
S31508005B6801D0204670BD214B1B78013BDBB23F2B89
S31508005B78F7D800F06DF81E4B18601E4B00221A70F5
S31508005B88194B01221A70ECE706460D46194B1B7885
S31508005B98013316481844FFF77FFF0446012815D134
S31508005BA8144B1A780132D2B21A70104B1B789A42E3
S31508005BB801D00024D5E710493046FFF767FC0A4BA1
S31508005BC800221A700B4B1B782B70CAE700F040F8B6
S31508005BD8074B1B686433984203D90024024B1C7090
S31508005BE8BFE70024BDE700BFA1120020601200200D
S31508005BF8A4120020A212002061120020024B0022E3
S31508005C081A605A609A60704710E000E008B5FFF716
S31508005C18F5FF054B054A5A6000229A600521196066
S31508005C28034B1A6008BD00BF10E000E0FF520700EA
S31508005C38A8120020044B1B6813F4803F03D0034ABC
S31508005C48136801331360704710E000E0A8120020BB
S31508005C5808B5FFF7EFFF014B186808BDA812002022
S31508005C6808B5FFF7F5FF08BD704772B6704762B604
S31508005C7870470A44914200F1FF3300D1704710B5C6
S31508005C8811F8014B03F8014F9142F9D110BD0000F4
S31508005C98F8B500BFF8BC08BC9E467047F8B500BF03
S30D08005CA8F8BC08BC9E467047D3
S31508005CB000000000000000000000000000000000D6
S31508005CC000000000010000000200000003000000C0
S31508005CD004000000000000000500000000000000AD
S31508005CE000000000000000000600000000000000A0
S31508005CF0000000000000000007000000000000206F
S31508005D00757362645F636F6E662E63006D61696E9C
S31508005D102E63000044656661756C740057696E559C
S31508005D2053422042756C6B20496E746572666163D6
S31508005D30650000004F70656E424C542055736572BD
S31508005D400000000057696E5553422042756C6B205F
S31508005D5044657669636500000100000002000000E2
S31508005D600400000006000000080000000A00000009
S31508005D700C00000010000000200000004000000099
S31508005D808000000000010000000102030405060768
S31508005D90080C10141820304000000000010203040B
S31508005DA001020304060708090000000001020304B3
S31508005DB001020304060708094F70656E424C540039
S31508005DC02E2E2F2E2E2F2E2E2F536F757263652F84
S31508005DD041524D434D375F53544D333248372F7533
S31508005DE073622E6300000000000002080000020033
S31508005DF00101000000000408000002000201000082
S31508005E000000060800000200030100000000080860
S31508005E10000002000401000000000A080000020059
S31508005E200501000000000C08000002000601000041
S31508005E3000000E080000020007010000000010081C
S31508005E400000020000020000000012080000020024
S31508005E50010200000000140800000200020200000F
S31508005E6000001608000002000302000000001808DF
S31508005E70000002000402000000001A0800000200E8
S31508005E800502000000001C080000020006020000CF
S31508005E9000001E0800000200070200002E2E2F2E0A
S31508005EA02E2F2E2E2F536F757263652F41524D4339
S31508005EB04D375F53544D333248372F63616E2E6327
S31508005EC0000000000502060206030703080309038B
S31508005ED009040A040B040C040C050D050E050F0530
S31508005EE00F061006100710082E2E2F2E2E2F2E2ED8
S31508005EF02F536F757263652F41524D434D375F536C
S31508005F00544D333248372F72733233322E630000C2
S30D08005F1021030008BD02000888
S30908005F1899020008D4
S31508005F1C00000000EC02002054030020BC03002003
S31508005F2C0000000000000000000000000000000057
S31508005F3C0000000000000000000000000000000047
S31508005F4C0000000000000000000000000000000037
S31508005F5C0000000000000000000000000000000027
S31508005F6C0000000000000000000000000000000017
S31508005F7C0000000000000000000000000000000007
S31508005F8C00000000000000000000000000000000F7
S31508005F9C00000000000000000000000000000000E7
S31508005FAC00000000000000000000000000000000D7
S31508005FBC00000000000000000100000000000000C6
S31508005FCC0E33CDAB34126DE6ECDE05000B0000008B
S31508005FDC00000000000000000000000000000000A7
S31508005FEC0000000000000000000000000000000097
S31508005FFC0000000000000000000000000000000087
S3150800600C0000000000000000000000000000000076
S3150800633C0000000000000000AC120020C10B000891
S3150800634CA90B0008490B000800000000000000001B
S3150800635C310B00083B0B00081D0B00080000000061
S3150800636C0000000000000000050B000800000000FB
S3150800637C110B000809022000010100C032090400B3
S3150800638C0002FF000000070581024000FF07050117
S3150800639C024000FF0A06000200000040010000004F
S315080063ACF90B0008050C0008B50C0008910C000840
S315080063BC7D0C0008D10C0008F50C0008120100022F
S315080063CC00000040501DAC600002010203010000F1
S315080063DC040309041A030000000000000000000072
S315080063EC0000000000000000000000000000010092
S315080063FC100000000090D0030090D00304000000A9
S70508000405E9
